:100000000C945B000C9461010C948E010C948300A1
:100010000C9483000C9483000C9483000C94830054
:100020000C9483000C9483000C9483000C94830044
:100030000C9483000C9483000C9483000C94830034
:100040000C94BB010C9483000C94C2030C948300A9
:100050000C9483000C9483000C9483000C94830014
:100060000C9483000C948300000024272A000025B0
:10007000282B000023262904040404040404040299
:100080000202020202030303030303010204081035
:100090002040800102040810200102040810200002
:1000A0000000070002010000030406000000000039
:1000B00000000000560111241FBECFEFD4E0DEBFC8
:1000C000CDBF11E0A0E0B1E0ECE5F8E002C00590A2
:1000D0000D92A831B107D9F711E0A8E1B1E001C054
:1000E0001D92A23BB107E1F710E0C6EBD0E004C0DF
:1000F0002297FE010E942804C43BD107C9F70E9441
:100100004F010C942C040C940000809108010E9473
:100110006E03892B09F08CC0809118019091190110
:10012000892B09F085C020910E0130910F0180913B
:100130000C0190910D01280F391F2F3F31053CF024
:100140008FEF90E090930D0180930C0104C03093E9
:100150000D0120930C0181E090E0909319018093B0
:10016000180104C0109219011092180180910A011F
:100170000E946E03892B09F063C080911A0190914F
:100180001B01892B09F05CC080910C0190910D013D
:1001900020910E0130910F01281739072CF0109291
:1001A0000D0110920C0106C0821B930B90930D0160
:1001B00080930C0181E090E090931B0180931A01E1
:1001C00004C010921B0110921A0160910C017091F1
:1001D0000D01809102010E94AD02809104010E94F4
:1001E0008F029093070180930601029734F482E016
:1001F00090E0909307018093060161E080910001F7
:100200000E94230362E070E080E090E00E942B02F5
:1002100060E0809100010E942303609106017091CB
:100220000701882777FD8095982F0E942B0208955B
:10023000809108010E946E03019709F097CF92CF39
:1002400080910A010E946E03019709F0BECFB9CFD9
:1002500061E0809100010E94050360E08091080147
:100260000E94050360E080910A010E94050361E09D
:100270008DE00E94050361E0809102010E94050368
:1002800061E0809108010E94230361E080910A01EE
:100290000E94230361E08DE00E94230308950E94E1
:1002A00055020E9428010E948500FDCF85E191E062
:1002B00090931D0180931C010895862F0E94BA031C
:1002C00008951F920F920FB60F9211242F933F9310
:1002D0004F935F936F937F938F939F93AF93BF934E
:1002E000EF93FF9380911E0190911F01892B29F0BC
:1002F000E0911E01F0911F010995FF91EF91BF91CF
:10030000AF919F918F917F916F915F914F913F91AD
:100310002F910F900FBE0F901F9018951F920F9264
:100320000FB60F9211242F933F934F935F936F93C8
:100330007F938F939F93AF93BF93EF93FF9380919E
:10034000200190912101892B29F0E0912001F09169
:1003500021010995FF91EF91BF91AF919F918F91ED
:100360007F916F915F914F913F912F910F900FBEB1
:100370000F901F9018951F920F920FB60F92112495
:100380002F938F939F93AF93BF938091220190916E
:100390002301A0912401B09125010196A11DB11D59
:1003A0008093220190932301A0932401B09325010F
:1003B0008091260190912701A0912801B0912901F7
:1003C0008050904CAF4FBF4F8093260190932701F0
:1003D000A0932801B093290127C080912601909114
:1003E0002701A0912801B091290180589E43A04087
:1003F000B0408093260190932701A0932801B093E9
:10040000290180912A0190912B01A0912C01B0919A
:100410002D010196A11DB11D80932A0190932B01FE
:10042000A0932C01B0932D0180912601909127017A
:10043000A0912801B091290181589E43A040B0406D
:1004400060F6BF91AF919F918F912F910F900FBE4A
:100450000F901F901895EF92FF920F931F937B01BF
:100460008C018FB7F89440912A0150912B01609133
:100470002C0170912D018FBF2FB7F89480912A0124
:1004800090912B01A0912C01B0912D012FBF841BC5
:10049000950BA60BB70BE816F9060A071B0760F7C2
:1004A0001F910F91FF90EF900895789484B582602A
:1004B00084BD84B5816084BD85B5826085BD85B508
:1004C000816085BDEEE6F0E0808181608083E1E8B7
:1004D000F0E0808182608083808181608083E0E8B9
:1004E000F0E0808181608083E1EBF0E080818460D6
:1004F0008083E0EBF0E0808181608083EAE7F0E0D8
:10050000808184608083808182608083808181603B
:1005100080838081806880831092C10008958F70ED
:10052000909110019295990F990F907C982B909330
:100530007C0080917A00806480937A0080917A00B8
:1005400086FDFCCF2091780040917900942F80E0C7
:1005500030E0282B392BC90108951F93CF93DF93E7
:10056000182FEB0161E00E940503E12FF0E0E15656
:10057000FF4F8491833051F4809180008068809394
:100580008000D0938900C09388003BC0843051F430
:1005900080918000806280938000D0938B00C09314
:1005A0008A002FC0813039F4209729F184B5806802
:1005B00084BDC7BD26C0823039F42097E1F084B5F0
:1005C000806284BDC8BD1DC0863041F48091B000FA
:1005D00080688093B000C093B30013C0873041F4AB
:1005E0008091B00080628093B000C093B40009C0D5
:1005F000C038D10514F460E001C061E0812F0E9491
:100600002303DF91CF911F910895282F30E0C90176
:1006100085579F4FFC01949129583F4FF9018491D0
:10062000882381F0E82FF0E0E859FF4FE491F0E0F3
:10063000662329F4808190958923808308958081A1
:10064000892B80830895482F50E0CA0181569F4F1F
:10065000FC012491CA0185579F4FFC019491495890
:100660005F4FFA0134913323C1F1222331F123305A
:1006700021F4809180008F7705C0243031F480917F
:1006800080008F7D8093800018C0213019F484B5DC
:100690008F7704C0223021F484B58F7D84BD0DC0D6
:1006A000263021F48091B0008F7705C0273029F4DF
:1006B0008091B0008F7D8093B000E32FF0E0E3598C
:1006C000FF4FE491F0E0662329F48081909589231F
:1006D000808308958081892B80830895482F50E07E
:1006E000CA0181569F4FFC012491CA0185579F4F33
:1006F000FC01949149585F4FFA013491332319F466
:1007000020E030E035C0222331F1233021F4809104
:1007100080008F7705C0243031F4809180008F7D78
:100720008093800018C0213019F484B58F7704C0FD
:10073000223021F484B58F7D84BD0DC0263021F494
:100740008091B0008F7705C0273029F48091B000E8
:100750008F7D8093B000E32FF0E0EE58FF4FE491DF
:10076000F0E0808120E030E0892311F021E030E0EA
:10077000C9010895982F8091C00085FFFCCF909308
:10078000C60008951F920F920FB60F9211242F9357
:100790003F934F935F936F937F938F939F93AF9309
:1007A000BF93EF93FF934091C600E0912E01F0912B
:1007B0002F01CF01019660E870E00E94FF039C01C9
:1007C00080913001909131012817390739F0EE5CA2
:1007D000FE4F408330932F0120932E01FF91EF9124
:1007E000BF91AF919F918F917F916F915F914F9149
:1007F0003F912F910F900FBE0F901F90189597FB70
:10080000092E07260AD077FD04D00CD006D0002090
:100810001AF4709561957F4F0895F6F7909581953C
:100820009F4F0895AA1BBB1B51E107C0AA1FBB1F06
:10083000A617B70710F0A61BB70B881F991F5A956C
:10084000A9F780959095BC01CD010895EE0FFF1F8B
:0C0850000590F491E02D0994F894FFCF7E
:10085C000200090004000A0011001300FF0014003C
:08086C0001000000005D010025
:00000001FF
